:020000040000FA
:06000000083002303A282E
:08000800A000030EA100831209
:100010008B1C32288B1031181428B11C3228643004
:10002000010203183128182800001628172818285C
:1000300019281A281B281C281D281E281F283110A3
:10004000B114A810031005190314AA0DA90DA80DC9
:10005000B00B322831152A08AF002908AE00280855
:10006000AD00B11081010B11210E8300A00E200EF6
:02007000090085
:0C007400203084008001840A6030040207
:10008000031C3C281230B00084218316FF2390000B
:10009000831283160C308505870183128501870141
:1000A000073099000030831691009F008312C830FA
:1000B00083168100831231309000003083168C004B
:1000C000831210308B00CA2181018E018F010B1128
:1000D0008B100B108C018B177C203119922068211A
:1000E000B30B7A28031085190314B90DF0303902C7
:1000F00003190421CF216C286400311808000B1D5E
:1001000008000B11B11031141230B000051D8D28FC
:10011000321483160113831208003210831601175C
:100120008312080031110130B7008B1320303707DC
:1001300083169B001C141A088312A400A500C0306B
:10014000A5061030370783169B001C141A0883126B
:10015000A3000030370783169B001C141A08831273
:10016000A2008B17321CBA2822090339A200A30966
:10017000A409A50922082D02031DFE2823082E022A
:10018000031DFE2824082F02031DD9280130370241
:10019000031DD028CF283D18D0283D143E14A0219F
:1001A00002303702031DD928BD18D928BD143E14CA
:1001B000A82125082F02031DF12801303702031D55
:1001C000E728E6283D1CE7283D103E14AB2102300D
:1001D0003702031DF028BD1CF028BD103E14B321CA
:1001E000FE285F08AB3C0319FE283218FA282F18A6
:1001F000FE28FD282F1CFE28FD28B621B70A033053
:1002000037020318080095280130B600B300B40087
:10021000B500B70085018701B113C3217C20B30B62
:100220003629031085190314B90DF030390203196A
:100230005D29B41F8501B41F8701B40B3629023034
:10024000370203192729B50B36290230B5000130D2
:1002500037020319B921023037020319BE21FA30DF
:10026000B4000230370296300319B400311D0E2954
:100270003111321C40292D090339AD00AE09AF09F7
:100280002F1CB1132F1C0E29B11B0E292E180E295D
:10029000B1178B1320303707BB002F08BA0071212C
:1002A00010303707BB002E08BA0071210030370725
:1002B000BB002D08BA0071218B17C621850187016B
:1002C000B70AB60103303702031C0E29CA21080001
:1002D0003E1C08003E101030BB003D08BA007121E2
:1002E00008008B133A0883161C159A003B089B00E4
:1002F00055309D00AA309D009C1464009C187D29F7
:100300001C1183128B170800831600309B001C14ED
:100310001A088312DF00831610309B001C141A0881
:100320008312BD00831620309B001C141A08831210
:10033000C1000130C11BC100C1080319C100080080
:10034000051205148E018F010C104108C000080031
:10035000851285140800051005168E018F010C10FA
:100360004108C00008008516851008000510051218
:100370000800380911398500B80008003809223909
:100380008500B8000800B80138140800B801B81496
:10039000B8160800BD188514BD1C851608000C1C75
:1003A0006C280C10C00B6C284108C0000510051209
:0203B000080043
:084000000A00030005000100A5
:02400E00CC01E3
:10420000010003000300030003000200020002009B
:1042100002000000000000000000FF00FF00FF009F
:10422000000000000000000000000000000000008E
:104230000000C000C000C000C000FF00FF00FF0081
:104240000100C300F300CF00FF00C300F300CF0064
:10425000FF00C300F300CF00FF00FF00FF00FF00DE
:10426000FF00FF00FF00FF00FF00FF00FF00FF0056
:10427000FF00FF00FF00FF00FF00FF00FF00FF0046
:10428000FF00FF00FF00FF00FF00FF00FF00FF0036
:10429000FF00FF00FF00FF00FF00FF00FF00FF0026
:1042A000FF00FF00FF00FF00FF00FF00FF00FF0016
:1042B000FF00FF00FF00FF00FF00FF00FF00FF0006
:1042C000FF00FF00FF00FF00FF00FF00FF00FF00F6
:1042D000FF00FF00FF00FF00FF00FF00FF00FF00E6
:1042E000FF00FF00FF00FF00FF00FF00FF00FF00D6
:1042F000FF00FF00FF00FF00FF00FF00FF00AA001B
:00000001FF
